:100000006E0A28001202B2022400080220006A0AC6
:10001000080C380017022400130254066109540723
:1000200063091502240056026709180243066A0A8A
:1000300014065109150224002B032A03000216019D
:100040000307960120002709F8021A0A6A0A170214
:1000500024001302A0010000A00100086D002C0084
:10006000FF0CEC010307ED0103076A0A030C2B00E8
:10007000DF0C3C09300A6B002A00E70CEA016B0236
:10008000FC0C0307470AEA010306430AEA010000E1
:10009000EB03430A0A064C0A2A07500A0000500ADA
:1000A00000082800A8026C006D005A0A2B032A03DE
:1000B0006C036D03E802560A0D022B000C022A00A5
:1000C0006A0A2001660AFF0F6001670AFF0F4701F5
:1000D00027000600C404A404000000086400FF0C0C
:1000E000270029000E0C3200FF0C2500C90409026C
:1000F000020007040702060027040702060047055E
:1001000007020600670507020600870407020600CB
:10011000A70407020600030C2D00E80C63002F095A
:10012000A604060586042605010C3900070C990073
:10013000A3040306A80A200CA601A70407020600D0
:10014000320C63002E09010CF901A3040307960A7F
:10015000030C2D00E80C63002F09010C630001095A
:10016000A3047C0BA604A3046607B80A6300B30AC1
:10017000020C63000109A304C50AA605A3046606D0
:10018000C30A6300BE0A6300AD0A0604060C35000C
:10019000100C3600060C3700020C3300010C340042
:1001A0006B00580C2A00100C630009096B00050C49
:1001B0002A00100C6300090906050604060C350028
:1001C000100C3600060C3700020C3300010C340012
:1001D0006B00950C2A00100C630009096B003C0CA5
:1001E0002A00100C6300090906050604060C3500F8
:1001F000100C3600060C3700020C3300010C3400E2
:100200006B006A00100C63000909040C2B00B30C8E
:100210002A00100C6300090906050604060C3500C7
:10022000100C3600060C3700020C3300010C3400B1
:100230006B006A00100C630009094E0C2B00420C85
:100240002A00100C630009090604060C3500100C86
:100250003600060C3700020C3300010C3400080C89
:100260002B006A00100C63000909800C2B00110C94
:100270002A00100C6300090906050604060C350067
:10028000100C3600060C3700020C3300010C340051
:100290006B00C40C2A00100C63000909800C2B00B1
:1002A000110C2A00100C6300090906057A00A3044A
:1002B0004606730B200CA601A70407020600BA022B
:1002C000050C63002E099A02A3044307710B200C4E
:1002D000A601A70407020600FA0C63002E096300BA
:1002E000630B6300570BA605D200F2002400000246
:1002F00028006400A305FB0B0604060C3500100C57
:100300003600060C3700020C3300010C34006B0081
:10031000580C2A00100C630009096B00050C2A0018
:10032000100C6300090906050604060C3500100CC4
:100330003600060C3700020C3300010C34006B0051
:10034000850C2A00100C630009096B002C0C2A0094
:10035000100C6300090906050604060C3500100C94
:100360003600060C3700020C3300010C34006B0021
:100370006A00100C63000909040C2B00B30C2A005E
:10038000100C6300090906050604060C3500100C64
:100390003600060C3700020C3300010C34006B00F1
:1003A0006A00100C630009094E0C2B00420C2A0055
:1003B000100C630009090604060C3500100C360009
:1003C000060C3700020C3300010C3400080C2B0023
:1003D0006A00100C63000909800C2B00290C2A000C
:1003E000100C6300090906050604060C3500100C04
:1003F0003600060C3700020C3300010C34006B0091
:100400007D0C2A00100C63000909800C2B00100CD5
:100410002A006300090906057A00A3054606290A91
:10042000200CA601A70407020600BA02050C63000F
:100430002E099A02A3054307270A200CA601A70448
:1004400007020600FA0C63002E09A305190AA3058A
:100450000D0AA604D200F200240000022800640065
:0C046000A305FB0BA305320AA305340A18
:0207EE00E8021F
:0E07F000F50BA304BD0AE802F90BA304B20A3C
:021FFE00EA0FE8
:00000001FF
